:03000000020347B1
:03000B00020648A2
:10001B00020659309306309403209204D209C2028F
:10002B00A2939213C21475240A12061F300304C242
:10003B0003D2052005030200D0A293120618200359
:10004B00030200D0C203C205C2090508E508B401CA
:10005B0009C2ABC213D2141205C6E508B40209C219
:10006B0013C214D2151205C8E508B4030BC213C290
:10007B0014C215D2161205CAE508B4040FD2ABC2CE
:10008B0013C214C215C216D2171205CCE508B4055B
:10009B000FC213C214C215C216C217D2181205CE44
:1000AB00E508B40613C213C214C215C216C217C296
:1000BB0018C219D21A1205D2E508B407081205C2E4
:1000CB00E4F508D202A2949213C21475240A120604
:1000DB001F300304C203D20620060302019012064E
:1000EB0016200303020190C203C206C209E508B43D
:1000FB00011B050EE50EB40A05E4F50E0511E5111D
:10010B00B4020AE50EB40405E4F50EF511E508B4E6
:10011B000216050DE50DB40A05050FE4F50DE50F07
:10012B00B40605E4F50DF50FE508B403160510E567
:10013B0010B40A050512E4F510E512B40605E4F552
:10014B0010F512E508B4041B0514E514B40A05E414
:10015B00F5140516E516B4020AE514B40405E4F526
:10016B0014F516E508B405160513E513B40A05E4F2
:10017B00F5130515E515B40605E4F513F515E508B6
:10018B00B40602B201A2929213C21475240A12068B
:10019B001F300304C203D207200703020250A292AE
:1001AB00120618200303020250C203C209C207E55C
:1001BB0008B4011C150EE50EB4FF05750E091511DB
:1001CB00E511B4FF0BE50EB40906750E03751102AC
:1001DB00E508B40217150DE50DB4FF05150F750DE8
:1001EB0009E50FB4FF06750D09750F05E508B40396
:1001FB00171510E510B4FF051512751009E512B4AB
:10020B00FF06751009751205E508B4041C1514E5F5
:10021B0014B4FF057514091516E516B4FF0BE51498
:10022B00B40906751403751602E508B40517151302
:10023B00E513B4FF051515751309E515B4FF067520
:10024B00130975150522300E1C850E27D213752840
:10025B000A75290D85112A850E2BD214AB117D0D34
:10026B007F0A120587300D1C850D27D21375280ABE
:10027B0075290B850F2A850D2BD214AB0F7D0B7FA8
:10028B000A120587300F1C851027D21375280A75A3
:10029B00290E85122A85102BD214AB127D0E7F0AE4
:1002AB00120587300C1C851427D21375280A752963
:1002BB000A752A0A752B0AC214AB167D0D7F0A121A
:1002CB000587300B1C851327D21375280A75290A4D
:1002DB00752A0A752B0AC214AB157D0B7F0A120502
:1002EB008730083820011975270CC21375280A7539
:1002FB00290A752A0A752B0AC2147B0CE4FD801798
:10030B0075270BC21375280A75290A752A0A752BCE
:10031B000AC214E4FB7D0A7F0A12058730111C8583
:10032B001327D21375280A75290A752A0A752B0A01
:10033B00D214AB15AD14AF1612058722787FE4F6F5
:10034B00D8FD75812F02038E02054EE493A3F8E4CA
:10035B0093A34003F68001F208DFF48029E493A312
:10036B00F85407240CC8C333C4540F4420C883402B
:10037B0004F456800146F6DFE4800B0102040810FA
:10038B0020408090049CE47E019360BCA3FF543F0B
:10039B0030E509541FFEE493A360010ECF54C02532
:1003AB00E060A840B8E493A3FAE493A3F8E493A322
:1003BB00C8C582C8CAC583CAF0A3C8C582C8CAC586
:1003CB0083CADFE9DEE780BEE517C394144005E47A
:1003DB00F5170510E510B40A050512E4F510E51242
:1003EB00B40607E4F510F512050DE50DB40A09E4A2
:1003FB00F510F512F50D050FE50FB4060BE4F5102E
:10040B00F512F50DF50F050EE50EB40A0DE4F5101A
:10041B00F512F50DF50FF50E0511E511B40212E508
:10042B000EB4040DE4F510F512F50DF50FF50EF500
:10043B001122E51165167058E50E65147052E50F23
:10044B006515704CE50D65137046D210C213C214BE
:10045B00C215C216C217C218D219C21A1205D2126D
:10046B0005F3209415D209A2949213C21475241487
:10047B0012061F300304C203D200300013120616FB
:10048B0030030DC203C209C200C210C2011205C063
:10049B0022011100010E00010F00010D00011200DD
:1004AB0001100001160001140001150001130001D9
:1004BB000800011700011800010900010A00010BD7
:1004CB0000010C00C103C184C10EC10DC10FC10CD1
:1004DB00C10BC108C111C100C101C102C110C10AC8
:1004EB00C109C112C105C106C10700E518B4040E4C
:1004FB00E4F5180509050A050B300902050CE5188A
:10050B00700BEF90066893F5B0D290D291E518B4CA
:10051B00010BED90066893F5B0C290D291E518B43B
:10052B00020BEB90066893F5B0D290C291E518B42C
:10053B00030CE52F90066893F5B0C290C291A215FB
:10054B009296221206331203D3E50BB43E05B20A80
:10055B00E4F50B30010630020312043D3004128522
:10056B000D2FA20A9215AB0FAD0EAF111204F68030
:10057B00031202512010CF12001E80CAE50AC39449
:10058B0032500A85272FA21392151204F6E50AC3DF
:10059B0094324016E50A94645010852B2FA21492C6
:1005AB0015AB2AAD29AF281204F6E50AC3946440B3
:1005BB0003E4F50A22C212D213C214C215C216C228
:1005CB0017C218C219C21AA2139204A214920EA235
:1005DB0015920DA216920FA217920CA218920BA2B3
:1005EB00199211A21A920822300A04A2129295E5CE
:1005FB0009C3943240050524E4F509E524B4640AE3
:10060B00E4F524C201C2101205C022A2949213D2A7
:10061B0014752405A213301401B3400BE50C95247B
:10062B004005D203E4F50C22758911D2AFD2A9D2C1
:10063B00ABC28DC28F75B808D28CD28E22C28CC23F
:10064B008D758CF8758A2FD28C0518B21232C28E2A
:10065B00C28F758D3C758BB6D28E0517323F06DB7C
:0D066B00CFE6EDFD07FFEF0037F1F6EDC023
:00000001FF
